:1000000000308A001A2B000000000A108A100A1122
:1000100082074C345A343434303431340D340034A3
:100020008316861083128614FF306500FB3066004D
:100030008830840080010808383981388800083009
:100040008D000808C7390D048800950194019701B7
:1000500096019A0114309100073092008316061120
:10006000831206152C2B08308C008316061483127D
:1000700006183828B3018C174B288C134B28031013
:10008000B30C0618B3170C174B280C138C0B3F2816
:1000900033088D0056281D308C1B07308D008D0BCA
:1000A0004F288C1B3D280C1B45283F280034950108
:1000B000940197019601B7011108370203183A29F4
:1000C00002306600B80112083802031878281908AF
:1000D000860005308C008C0B6B2800000000063079
:1000E000860003308C008C0B73283808B80A63280C
:1000F0000000000000000000000000000E3086003C
:10010000063086000815081983280908B900F3305D
:100110006600A2013908A1002108960722080318E9
:10012000013E970713308C008C0B942800000000D0
:1001300002306600B801120838020318B028190806
:10014000860005308C008C0BA328000000000630D0
:10015000860003308C008C0BAB283808B80A9B282B
:1001600005308C008C0BB2280E30860006308600DD
:1001700008150819B9280908B900F33066009C0170
:1001800039089B001B0894021C08031C9503950268
:1001900013308C008C0BCA2800000000023066006F
:1001A000B801120838020318E6281908860005303D
:1001B0008C008C0BD928000000000630860003302C
:1001C0008C008C0BE1283808B80AD12808308C0044
:1001D0008C0BE82800000E308600063086000815DB
:1001E0000819F0280908B900F33066009E013908A3
:1001F0009D001D0896021E08031C970397021330EA
:100200008C008C0B01290000000002306600B80150
:100210001208380203181D291908860005308C00C1
:100220008C0B1029000000000630860003308C0083
:100230008C0B18293808B80A08290B308C008C0B55
:100240001F29000000000E308600063086000815C9
:10025000081928290908B900F3306600A0013908F7
:100260009F001F08940720080318013E95073708D0
:10027000B70A5C28FB3066001C082002031C4829D2
:100280001C082002031D55291B081F0203185529AD
:100290008D00FF308C0014080C029400FF308C009D
:1002A0001508031C8C030C0295001E082202031C77
:1002B00061291E082202031D6E291D082102031850
:1002C0006E298D00FF308C0016080C029600FF305E
:1002D0008C001708031C8C030C0297001608940767
:1002E00017080318013E950700348030B50006302A
:1002F000350799001A08B40004301A0734020318AD
:100300009929572034088C0003108C0D0C088C00A0
:1003100023300C0784001508840A80008403140825
:1003200080000310B50C0630350799003408B40A74
:100330007C29003408308D008316061183120611C3
:100340008D17AF298D13B50C03180615031C061164
:100350000D17AF290D138D0BA3290615AF291D30DD
:100360008400840BB1298D1BA2290D1BAA290034FE
:100370001A08B30004301A0733020318E1293308BE
:100380008C0003108C0D0C088C0023300C078C00A3
:1003900001300C0784000008B4003408B5009A212D
:1003A00033088C0003108C0D0C088C0023300C07D4
:1003B00084000008B4003408B5009A213308B30A59
:1003C000BA29352B08308D008316861083128610CB
:1003D0008D17F7298D13BA0C03188614031C861089
:1003E0000D17F7290D138D0BEB298614F7291D30F6
:1003F0008400840BF9298D1BEA290D1BF229003496
:100400001A08B30004301A0733020318292A3308E4
:100410008C0003108C0D0C088C0023300C078C0012
:1004200001300C0784000008B4003408BA00E2214F
:1004300033088C0003108C0D0C088C0023300C0743
:1004400084000008B4003408BA00E2213308B30A7B
:10045000022A3B2B8D018E018C018F013D08031D6B
:10046000342A3C0803194E2A1030BE000310BA0D7E
:10047000BB0D8C0D8F0D3D080F02031D412A3C085A
:100480000C02031C4A2A3C088C02031C8F033D0803
:100490008F0203148D0D8E0DBE0B362A0000003422
:1004A0003708BB003608BA002730BD001030BC004A
:1004B0002A2230300D07B8000E08B9000318B90A17
:1004C0003808BA00E2213708BB003608BA0003300A
:1004D000BD00E830BC002A220E08BB000D08BA009F
:1004E000BD010A30BC002A220C088C0030300C07F9
:1004F000B8000F08B9000318B90A3808BA00E22199
:100500003708BB003608BA00BD016430BC002A229F
:100510000E08BB000D08BA00BD010A30BC002A223B
:100520000C088C0030300C07B8000F08B900031815
:10053000B90A3808BA00E2213708BB003608BA0009
:10054000BD010A30BC002A220E08BB000D08BA000B
:10055000BD010A30BC002A220C088C0030300C0788
:10056000B8000F08B9000318B90A3808BA00E22128
:100570003708BB003608BA00BD010A30BC002A2289
:100580000C088C0030300C07B8000F08B9000318B5
:10059000B90A3808BA00E22100341A08B30003305F
:1005A0001A0733020318EE2A33088C0003108C0D4F
:1005B0000C088C0023300C078400840A0008840394
:1005C000B5000008B4003508B7003408B600502262
:1005D0002030BA00E2213308B30ACF2A33088C0056
:1005E00003108C0D0C088C0023300C078400840A47
:1005F00000088403B5000008B4003508B7003408CB
:10060000B60050220D30BA00E22100347521CD220F
:10061000003408308D000808C7390D0488009A019D
:10062000003410308D000808C7390D0488000430EC
:100630009A000034840188308400073080008316DB
:1006400086108312861483160611831206158316EC
:10065000861083128614102833200D089800553018
:100660001802031D352B7521B82959301802031DB6
:100670003B2B7521002A57301802031906235230EC
:100680001802031D482B09230623112306239A0170
:1006900053301802031D552B57201508B7001408B6
:1006A000B60050220D30BA00E22143301802031D7B
:1006B0006E2B33200D08980030301802031D662B76
:1006C00000308D000808C7390D0488003130180249
:1006D0000319092332301802031911235830180264
:1006E000031D8D2B33200D08980030301802031D98
:1006F0007B2B8630990031301802031D812B463048
:10070000990032301802031D872B263099003330B0
:100710001802031D8D2B1630990054301802031D4A
:10072000D82B110893000130910057201A088C0033
:1007300003108C0D0C088C0023300C078400220859
:10074000840A800084032108800001301A078C008D
:1007500003108C0D0C088C0023300C0784001C083F
:10076000840A800084031B08800002301A078C0072
:1007700003108C0D0C088C0023300C0784001E081D
:10078000840A800084031D08800003301A078C004F
:1007900003108C0D0C088C0023300C0784002008FB
:1007A000840A800084031F088000CD221308910072
:1007B00049301802031DE22B33200D08910033202D
:1007C0000D08920056301802031DF02BB3013308B8
:1007D0000520B30ABA00E22106303302031DE72BDD
:0807E000FB3066002C2B6300C6
:02400E00FA3F77
:00000001FF
